:1000000023EF00F0EA6A060EE96EEF500DE0060EEF
:10001000016E006A002EFED7012EFBD77B0E006E0C
:10002000002EFED7EF2EF3D75BEF00F0030E065E37
:1000300009E3EA6A060EE96EEF5004E001D000D051
:10004000EF2EFDD7000CF86AD09EEA6AE96AC1502B
:10005000C00B0F09C16E070EB46EC150C00B0F0963
:10006000C16EC090C092C094C09EC2809698C69A3D
:10007000949E93809392010EC66E000EC76ED1902F
:10008000800ED56ECD6A000ECA6E000ECB6EB16AC0
:10009000070EB46E9250926E100E006E002EFED7B8
:1000A0000000B450A19CB56A96908D90040E056E28
:1000B000FA0E066EA7D7052EFBD796908D80A60E5A
:1000C000006E002EFED7000096908D70040E056E17
:1000D000EA0E066EABDF052EFBD796908D70A60E4E
:1000E000006E002EFED7000096908D70040E056EF7
:1000F000EA0E066E9BDF052EFBD796908D70A60E3E
:10010000006E002EFED7000096908D70040E056ED6
:10011000EA0E066E8BDF052EFBD796908D70C80E0B
:10012000066E84DF96908D70A60E006E002EFED7B0
:10013000000096908D70A60E006E002EFED7000077
:1001400096908D70A60E006E002EFED70000969041
:100150008D70A60E006E002EFED7000096908D705A
:10016000A60E006E002EFED7000096908D70C80E71
:0E017000066E5CDF96908D7097D7FFD7030068
:020000040030CA
:0E00000027CC380E008780000FC00FE00F40A5
:00000001FF
